:100000002038001023B80000CF800012CC000085FB
:1000100004180001CD80000ECD800083CC0000824A
:10002000CD800081CC00000B8000004A0000000061
:10003000CC00000ECC00000EC8100082202801C3A6
:10004000201C0000C8100082C80800857F8B800734
:10005000C808008194800030000000008000005437
:1000600000000000C9CC008394C00017000000000D
:1000700084000097200C0001840000AA20380000B2
:1000800097800011200C000DC0302009CCF1000039
:10009000C030200AC03418181374000823741818CC
:1000A000CB0D00007CF4C006C808001A988000063A
:1000B000201C000194C0FFFB0000000080000041F4
:1000C0007DC1C006840000BD11B8001F840000AAD5
:1000D0002038000184000097200C0000C03001C0CF
:1000E000CB3900002038000095C0FFD3CF8000033B
:1000F0007DC1C006840000BD203800008000000DD6
:10010000CF80000320380001CF800003C810008298
:10011000CC000081C808001A9480000E0000000086
:10012000CD80000E00000000840000A820380002EE
:10013000CC310000840000AA20380001CD8000816D
:1001400084000097200C00008000000D00000000DB
:10015000C83800569B80006B201C0000C838005730
:100160009B800068201C0001201C0000C808008142
:100170009480001200000000C82800009680000F44
:1001800020080001CD80000ECC8000001C1C000067
:100190002A8801BB9480000400000000800000B8A1
:1001A000000000002A8801BC988000440000000084
:1001B0009500002300000000C82800029680000679
:1001C00020080001CD80000ECC8000028000008F4E
:1001D00000000000C8280001968000070000000011
:1001E00020080001CD80000ECC8000018000008F2F
:1001F00000000000C82800039680000900000000ED
:10020000CD80000E2A8C01E598C0FF9720080001E0
:10021000CC8000038000008F00000000C82800048C
:100220009680FF850000000020080001CD80000EB0
:10023000CC8000048000008F000000008400009348
:10024000000000008000000D000000001EA800FF5C
:10025000CE80000C8800000000000000C030039039
:10026000CB390000C00BFFFE7F8B800610CC001046
:100270007F8F8007CFB1000088000000CB390000DD
:10028000CFB10000CD80000ECB39000017B80004BC
:100290009780FFFE000000008800000000000000C2
:1002A000800000A0C03001C1C0302003CFB10000E9
:1002B00088000000CB390000C9F800839B8000044F
:1002C000000000008000000D00000000CC1C008336
:1002D000840000BD11B8001F8000000D0000000068
:1002E000CD9C0083840000BD203800009500FF54A1
:1002F00000000000C03001C088000000CFB1000045
:1003000099C0000BC830004023300002CF000040ED
:10031000840000D520380003C83000401F3003FDA2
:10032000CF00004080000054CC000056C830004090
:1003300023300040CF000040840000E62038000158
:10034000C83000401F3003BFCF0000408000005481
:10035000CC000056840000F100000000C0302008EE
:10036000840000F92038FFFFC0302008CC310000A5
:10037000CB390000C0300398840000F92038010018
:10038000C0300398CC310000CB090000C03021B64A
:1003900088000000CC310000840000F10000000063
:1003A00020380001C0300398840000F913B800140D
:1003B000CC000057C0300398CC310000880000000A
:1003C000CB090000CF9C0016CD80000EC9F00018AC
:1003D0007F38800C9480FFFE000000008800000041
:1003E00000000000CFB10000CB3900002008001F42
:1003F0009880000008880001CC1C0016C9F0001B82
:100400009700FFFF000000008800000000000000CF
:1004100000000000000000000000000000000000DC
:1004200000000000000000000000000000000000CC
:1004300000000000000000000000000000000000BC
:1004400000000000000000000000000000000000AC
:00000001FF
